:040000008031112812
:10000800803120007F08F4000B1C0D28803113205C
:100018000B1074082000FF0009008031AD2827006C
:10002800931D3E2820008C192328302822008C1686
:100038000530F100F10B1E2822008C123028803187
:10004800B5208031003A03191A28013A03193028DB
:10005800033A0319302830280530F3000F30F20036
:10006800F430F100F10B3628F20B3628F30B362862
:1000780027009311131E080020000C1E462880310B
:100088008F2080310530F3000F30F200F430F1009A
:10009800F10B4C28F20B4C28F30B4C2827001312B9
:1000A8000800033023008C008E0122001D1321005C
:1000B8008C1222008C1221000C1122000C1121003C
:1000C8008E1122008E1121000E1222000E12210024
:1000D8008E1222008E1221008C150C168C140C1412
:1000E8000E118E100E100800210099171908873973
:1000F80070389900FC309905803155208031803165
:10010800A62080318031B72080318031B220803103
:10011800F501F6018E289A28F501F50A0800023043
:10012800F0007008F5000800F50108007508003AAD
:1001380003199028013A03199328033A03199828B8
:10014800982808008B15270091159215111612167C
:100158000800F501F6012000803178280B178B176D
:080168000800750808000800FA
:020000040001F9
:04000E00A4FFFFDF6D
:00000001FF
